:020000040000FA
:08000000803102288731ED2F49
:100B8A00FE0012001E00FE0BC62D0034063405348A
:100B9A00033402340134073408340434F200EB2DF0
:100BAA00FC30132E6030132EDA30132EF230132E4F
:100BBA006630132EB630132EBE30132EE030132EAD
:100BCA00FE30132EF630132E0030132E7208F0006A
:100BDA00F1017108003A0319F32DE92D7008003A62
:100BEA000319D52D013A0319D72D033A0319D92D23
:100BFA00013A0319DB2D073A0319DD2D013A0319CE
:100C0A00DF2D033A0319E12D013A0319E32D0F3AB7
:100C1A000319E52D013A0319E72DE92D0800F20021
:100C2A00F301F601F7017208F0007608073C890A19
:100C3A001F2EF036890B1E2E701C242E252E362EC2
:100C4A000130F0007608203E860087010108FF3E49
:100C5A00890A302EF035890B2F2E7008F1007108A1
:100C6A00F3040130F6070030F73D7708803AF000C8
:100C7A0080307002031D432E08307602031C462E74
:100C8A00472E182E0730F4000030F5007308F000E4
:100C9A00740A502EF036890B4F2E7018552E582E86
:100CAA0020008E155A2E20008E110E160E12FF30BD
:100CBA00F407FF30F53DF51F632E642E4B2E8E117F
:100CCA000800F601F31F6A2E6B2E722EF209F30941
:100CDA00F20A0319F30AF601F60AF11F752E762EA7
:100CEA007B2EF009F109F00A0319F10A7008710460
:100CFA000319802E812EAA2EF501F50A8D2E0130B8
:100D0A00F035F10D890B852E0130F4007408F507D2
:100D1A00F11F902E912E842E71087302031D972EB7
:100D2A0070087202031C9A2E9B2E9F2E7008F202E4
:100D3A007108F33B0130F136F00C890BA02E01301B
:100D4A00F502031DA92EAA2E912E76080319AE2E9E
:100D5A00AF2EB42EF209F309F20A0319F30A730843
:100D6A00F1007208F00008002100191599111916EE
:100D7A0099161E169E121E179E130C1623000C1689
:100D8A0021001D159D151D129D121D131D140E11F6
:100D9A008E110E128E1223000E118E1120008E1249
:100DAA000E1121009D149D18DB2EDC2ED82E1C3628
:100DBA00F8007808FB0020008E160E160E128E120E
:100DCA000E160E128E160E160E120E150E160E1286
:100DDA000E110E160E12F901FA017B18F52EF82ED5
:100DEA0020008E15FA2E20008E110E160E127B0888
:100DFA00F8000130F836890BFF2E7818052F082FD6
:100E0A0020008E150A2F20008E110E160E127B0856
:100E1A00F8000230F836890B0F2F7818152F182F83
:100E2A0020008E151A2F20008E110E160E127B0826
:100E3A00F8000330F836890B1F2F7818252F282F32
:100E4A0020008E152A2F20008E110E160E127B08F6
:100E5A00F8000430F836890B2F2F7818352F382FE1
:100E6A0020008E153A2F20008E110E160E127B08C6
:100E7A00F8000530F836890B3F2F7818452F482F90
:100E8A0020008E154A2F20008E110E160E127B0896
:100E9A00F8000630F836890B4F2F7818552F582F3F
:100EAA0020008E155A2F20008E110E160E128E1546
:100EBA000E160E128E110130F9070030FA3D7A082B
:100ECA00803AF80080307802031D6D2F04307902D1
:100EDA00031C702F712FF22E20000E150E118E1684
:100EEA000E160E128E120E160E128E160E160E12E8
:100EFA000E160E120E160E128E120A30F000003066
:100F0A00F1007C080B3EF200003003180130F300B8
:100F1A0086316626863170088531D3258631863139
:100F2A00142686310A30F0000030F1007C08063EB3
:100F3A00F200003003180130F3008631662686314C
:100F4A0070088531D32586318631142686310A30D8
:100F5A00F0000030F1007C08043EF2000030031873
:100F6A000130F30086316626863170088531D32533
:100F7A0086318631142686317C088531D32586311F
:100F8A0086311426863120000E150E110130A8076D
:100F9A000030A93D2908803AF80080307802031D04
:100FAA00D82F64302802031CDB2FDC2FD62E20001A
:100FBA00A801A9010130F8007808FC070A307C0270
:100FCA00031CE82FE92FD62EFC01D62E80310228E9
:100FDA00CB308400853085002030860000308700C1
:100FEA0008308531C5258731FB01FC01A801A9011B
:060FFA0020008631B92E33
:020000040001F9
:04000E00A4C9CFDFD3
:00000001FF
